:040000008A01BD288C
:08000800F500F50E030EF600F1
:10001000040EF7000A0EF8008A110A12E128EE29F0
:10002000142A5D2ADB2ADF2AB02B1C2C832CC62C39
:10003000202D672D7A2DC72DE22D432E972E482F88
:10004000A22F8A150A1269288A150A1297298A1579
:100050000A12A2298A150A12C4298A150A12DB2952
:100060008A150A12112A8A150A122F2A8A150A12CB
:10007000502A8A150A12602A8A150A126A2A8A15D3
:100080000A12822A8A150A12982A8A150A12FE2A48
:100090008A150A12552B8A150A12852B8A150A12FF
:1000A000DE2B8A150A12FB2B8A150A121B2C8A15C5
:1000B0000A12512C8A150A12762C8A150A129A2CC9
:1000C0008A150A12A42C8A150A12BB2C8A150A1248
:1000D000F52C8A150A12822D8A150A12002E8A150D
:1000E0000A12212E8A150A12322E8A150A123F2E62
:1000F0008A150A12502E8A150A125D2E8A150A12C6
:100100006A2E8A150A12772E8A150A12852E8A15EA
:100110000A12932E8A150A12A02E8A150A12AE2EE2
:100120008A150A12BD2EFA0000308A009C307A0728
:1001300003188A0A7A0882070E308A00E62E0E30EB
:100140008A00FF2E0F308A00182F0F308A00312FBF
:100150000F308A004A2F0F308A00632F0F308A0039
:100160007C2F0F308A00952F0F308A00AE2F0F3072
:100170008A00C72F0F308A00D82F83120313D501AE
:100180002030D6001D208A110A125D208A110A1221
:1001900060208A110A12003C0319D228FF30831212
:1001A0000313CC0012208A110A120F208A110A129E
:1001B000033083120313C5006C208A110A128B17B7
:1001C000DF28831203134A08490201300318030190
:1001D0008316B6000B080439003C031931290B11B2
:1001E000203083125302013003180301D30A003C6C
:1001F00003190229780E8A00770E8400760E830098
:10020000750E0900D3014C08FF3C013003190301AE
:10021000FF39031D0F294D08FF390319102901303B
:10022000FF39031D1A29CE080130031D0301FF39D0
:1002300003191B290130003C03192F2966208A115C
:100240000A12831203133708BA003808BB003908B2
:10025000BC003408BD003508BE003608BF001F14BE
:100260001F15831203130C084039003C03195A2947
:100270000C131F101E08CA00410883163602031D06
:10028000552983124008831636020319552936086A
:100290008312C00083163608031952291A208A11C6
:1002A0000A12552919208A110A12831603133608D7
:1002B0008312C1000B080139003C031979290B1086
:1002C00063208A110A1283160313B7003708031933
:1002D000702937088312E80021208A110A1279292F
:1002E00060208A110A12003C0319792920208A1102
:1002F0000A12831203134C08F0007008013C031D1E
:10030000852915208A110A12E6297008023C031D6E
:10031000902913208A110A1213208A110A12E62941
:100320007008FF3C031DE22983120313CE0801303D
:10033000031D0301003C0319A12914208A110A128C
:10034000E629831203134D08F1007108003C031DD8
:10035000AD2916208A110A12E1297108013C031DFA
:10036000B52917208A110A12E1297108023C031DE0
:10037000BA29DC297108033C031DBF29DC29710857
:10038000043C031DC429DC297108053C031DC9294F
:10039000DC297108063C031DCE29DC297108073CC5
:1003A000031DD329DC297108083C031DD829DC2949
:1003B0007108093C031DE02911208A110A12E12964
:1003C000E129E62918208A110A12E629780E8A0006
:1003D000770E8400760E8300750E090039208A118D
:1003E0000A1283160313A601A7013F208A110A12DD
:1003F00083120313C20157208A110A1283160313B2
:10040000A6010130A7003F208A110A12033083128F
:100410000313C20057208A110A1283160313A50181
:100420003C208A110A120800831203133A0883162B
:10043000AF0051208A110A122E3083160313AA002E
:100440004B208A110A123B088316AF0051208A11F3
:100450000A122E3083160313AA004B208A110A12A7
:100460003C088316AF0051208A110A1220308316EF
:100470000313AA004B208A110A1220308316AA0007
:100480004B208A110A1220308316AA004B208A11B1
:100490000A123D088316AF0051208A110A123A3021
:1004A00083160313AA004B208A110A123E088316F2
:1004B000AF0051208A110A12080002308312031380
:1004C0004D02FB000830FC0072208A110A12F20073
:1004D0007C08003EF3000318F20A7308831203132A
:1004E000D7008316A601A7013F208A110A12063001
:1004F00083120313C20057208A110A120B3083168D
:100500000313A600A7013F208A110A12F20131301D
:10051000F3000230831203134D0273070318F20A2B
:100520008316AA004B208A110A128316A6010130F5
:10053000A7003F208A110A1283120313570883165B
:10054000AD000830AE004E208A110A120930831225
:10055000C20057208A110A12831203134E0803198E
:10056000CC2A01304E028316A6000130A7003F209E
:100570008A110A128312031352088316AA004B2011
:100580008A110A1201304E028316A6000130A7001C
:100590003F208A110A12D32A83160313A601A7014A
:1005A0003F208A110A12013083160313A5003C2054
:1005B0008A110A12080042208A110A1208008312C6
:1005C00003134808FB000830FC0072208A110A124D
:1005D000F1007C08003EF2000318F10A7208831251
:1005E0000313D8008316A5013C208A110A12831236
:1005F00003135108E5001E208A110A128316A60172
:10060000A7013F208A110A128312031320088316C0
:10061000AF0051208A110A122E3083160313AA004C
:100620004B208A110A1221088316AF0051208A112B
:100630000A122E3083160313AA004B208A110A12C5
:1006400022088316AF0051208A110A122030831627
:100650000313AA004B208A110A1258088316AD0012
:100660000430AE004E208A110A122030AA004B201E
:100670008A110A12F10151084F02013E0318F10AD2
:100680008316AF0051208A110A1283160313A601A4
:100690000130A7003F208A110A1283120313230896
:1006A0008316AF0051208A110A123A3083160313C1
:1006B000AA004B208A110A1224088316AF00512089
:1006C0008A110A122D3083160313AA004B208A11B7
:1006D0000A1225088316AF0051208A110A123A30F7
:1006E00083160313AA004B208A110A1226088316C8
:1006F000AF0051208A110A128312031327088316B0
:10070000AF0051208A110A122E3083160313AA005B
:100710004B208A110A1228088316AF0051208A1133
:100720000A120B3083160313A6000130A7003F20E6
:100730008A110A12203083160313AA004B208A1153
:100740000A120E308316A600A7013F208A110A1252
:10075000013083160313A5003C208A110A120800F9
:1007600083160313A601A7013F208A110A128312E0
:1007700003134D08F1007108003C031DC32B162024
:100780008A110A120D2C7108013C031DCB2B172076
:100790008A110A120D2C7108023C031DD02BF22B7A
:1007A0007108033C031DD52BF22B7108043C031D7B
:1007B000DA2BF22B7108053C031DDF2BF22B71089D
:1007C000063C031DE42BF22B7108073C031DE92BAB
:1007D000F22B7108083C031DEE2BF22B7108093C2B
:1007E000031DF62B11208A110A120D2C0C308312D6
:1007F0000313C20057208A110A1283160313A6019D
:100800000130A7003F208A110A120F308312031310
:10081000C20057208A110A120D2C83160313A60159
:10082000A7013F208A110A12013083160313A50085
:100830003C208A110A120800831203134B08FB00A4
:100840000830FC0072208A110A12F1007C08003E78
:10085000F2000318F10A720883120313D9008316F9
:10086000A601A7013F208A110A1210208A110A123C
:1008700083160313A6010130A7003F208A110A1234
:100880008312031359088316AD000830AE004E20C2
:100890008A110A122030AA004B208A110A12F6305F
:1008A0008316AA004B208A110A1220308316AA0050
:1008B0004B208A110A124B08E3001C208A110A12ED
:1008C00027088316AF0051208A110A122E30831692
:1008D0000313AA004B208A110A1228088316AF00BE
:1008E00051208A110A1283160313A6010130A700B2
:1008F0003F208A110A12013083160313A5003C2001
:100900008A110A1208000130831203134E02FB0001
:100910000330FC0072208A110A12F2007C08831254
:100920000313DA008316A601A7013F208A110A12D9
:10093000123083120313C20057208A110A12831641
:100940000313A6010130A7003F208A110A121020CC
:100950008A110A12831203135A08063C0318B62C94
:10096000F2015A08023E0318F20ADA005A08831606
:10097000A6000130A7003F208A110A120130831619
:100980000313A5003C208A110A12080083160313E2
:10099000A601A7013F208A110A1215308312031302
:1009A000C20057208A110A1283160313A6010130D0
:1009B000A7003F208A110A12183083120313C200C5
:1009C00057208A110A12043083160313A60001303F
:1009D000A7003F208A110A123A3083160313AA0097
:1009E0004B208A110A1249088316B00054208A113C
:1009F0000A120C3083160313A6000130A7003F2013
:100A00008A110A123A3083160313AA004B208A1166
:100A10000A124A088316B00054208A110A120530BF
:100A200083160313A6000130A7003F208A110A1283
:100A3000013083160313A5003C208A110A12080016
:100A4000831203134B08FB000830FC0072208A114C
:100A50000A12F1007C08003EF2000318F10A720845
:100A600083120313DB008316A601A7013F208A111E
:100A70000A1210208A110A1283160313A6010130EC
:100A8000A7003F208A110A12831203135B08831602
:100A9000AD000830AE004E208A110A1283124008C1
:100AA000003C0319592D1B30C20057208A110A122D
:100AB000602D1E3083120313C20057208A110A12C0
:100AC00083160313A5013C208A110A120800831221
:100AD00003134F08E5001E208A110A123D08A500E5
:100AE0003E08A6004B08C8004F08E6001F208A11E8
:100AF0000A120800831203134F08003C0130031D43
:100B00000301F0005008003C0130031D0301700593
:100B1000003C03198D2DD00AA02DF0014F08013E95
:100B20000318F00A50020319972D00309C2D70080D
:100B3000003C0130031D0301003C0319A02DD00A25
:100B4000CF0A4030EA004F08EB0027208A110A1232
:100B5000413083120313EA005008EB0027208A116A
:100B60000A12831203133A08A0003B08A1003C08B4
:100B7000A2003D08A3003E08A400A501A6014B0861
:100B8000C8004F08E6001F208A110A1208008312CD
:100B900003135C08F100F10CF10CF10CF10CF10CF9
:100BA000710C03390339FE005C08F100F10D710D81
:100BB000FC39FC39FF00F1017E081C3E0318F10AE4
:100BC000FE00080083120313DD01DE013A08DF0096
:100BD0003B08E0003C08E1004F08E2006208E50045
:100BE0001E208A110A12630848020130031D030106
:100BF000FF390319042E20085F020130031D030191
:100C0000FF390319042E0130FF390319102E210872
:100C100060020130031D0301FF390319102E01305A
:100C2000FF3903191C2E220861020130031D030144
:100C3000FF3903191C2E0130003C0319372EF10136
:100C40005D08F200270872070318F10ADD00F101C0
:100C50005E08F200280872070318F10ADE003C3033
:100C60005E02031C372E3C305E02DE00DD0A6208A5
:100C70005002031D3C2E3E2EE203EE2D5D08A70020
:100C80005E08A80008000E30831603139F00413051
:100C900083129F0082308316810001308500E0308E
:100CA0008600870183128601CC01C001C101C20107
:100CB000CD01CE01CA01D4014330E90024208A11BC
:100CC0000A120313CB004030E90024208A110A12D3
:100CD0000313CF004130E90024208A110A120313C4
:100CE000D0004230E90024208A110A120313C900FF
:100CF00066208A110A12831203133708BA003808D3
:100D0000BB003908BC003408BD003508BE003608F9
:100D1000BF000C130B1083160C170B178B158112C9
:100D200001120114811401150B118B1608000730F4
:100D300083120313E4006508DC001B208A110A12E9
:100D4000F1017F08033E0318F10AFF007E08EC0062
:100D50007F08ED002A208A110A122A08F10064088F
:100D6000E403293E84007108831380008312031377
:100D70002908F1006408E403293E84007108831304
:100D80008000FF30831203136402031DC82ECF2E90
:100D90007F08013CF1007109013EFF00A62E2908E1
:100DA0001F39A0002A080F39A1002908F100710C91
:100DB0007F391039F1002A08F200F20CF20CF20C23
:100DC000720C0F390F397104A2002B081F39A300D0
:100DD0002C083F39A4002D081F39A5002E083F39E3
:100DE000A6002D08F100F10CF10C710C1F3904392B
:100DF000F1002E08F200F20CF20CF20CF20CF20CE4
:100E0000720C033903397104C8004008FF39031913
:100E1000122F65084F020130031D0301FF3903192A
:100E2000122F0130003C03191B2F3D08A5003E087E
:100E3000A6004B08C8002508F10023087102A7008E
:100E40002608F10024087102A8002508F1002308F3
:100E500071020318332FF1011830F20027087207CE
:100E60000318F10AA7002608F100240871020318EC
:100E7000472FF1013C30F200280872070318F10AED
:100E8000A8002708013CF1007109013EA7000800F5
:100E9000831203132208F000F00D700DFC39203985
:100EA000F00020081F397004A9002208F000700E1D
:100EB000F039F039F039F00021080F397004AA0038
:100EC0004808F000F00DF00D700DF8392039F000F1
:100ED00023081F397004AB004808F000F00DF00D36
:100EE000700EF039C039C039F00024083F39700461
:100EF000AC004808F000F00DF00D700DF839203905
:100F0000F00025081F397004AD004808F000F00D0E
:100F1000F00D700EF039C039C039F00026083F39A5
:100F20007004AE00AF01B0016608DC001B208A111E
:100F30000A127E08EF007F088316A0002D208A1178
:100F40000A12080083120313E701FF304C02031951
:100F5000C12F831203134F08D10001304C02031D2F
:100F6000B82F4330EA004B08EB0027208A110A1201
:100F700083120313CC0A4C08023C0318C02FCC0187
:100F80000800CE0A4D08F0007008003C031DDE2F5B
:100F9000831203134E08053C0318DD2FCE013A08D7
:100FA000B7003B08B8003C08B9003D08B4003E0853
:100FB000B500B60169208A110A1208007008013CC8
:100FC000031DF12F831203134E08013C0318F02F69
:100FD000CE014230EA004908EB0027208A110A12AC
:100FE00008007008023C031DF82F8A150A122028F9
:100FF0007008033C031DFF2F8A150A122028700871
:101000008A150A12043C8A150A12031D0828202892
:101010007008053C031D0D2820287008063C031DA0
:10102000122820287008073C031D17282028700864
:10103000083C031D1C2820287008093C031D632858
:10104000F1018312031367084E070318F10AE70042
:1010500001306702013CF1007109013EE7000230F6
:101060004D02FB000830FC008A110A1272208A151A
:101070000A12F1007C08831203136707F2000318B9
:10108000F10A7208E7004E08013C0318502867086F
:10109000EA005208EB008A110A1227208A150A1268
:1010A000831203134E08083C03185828CE01682801
:1010B000E70A6708E9008A110A1224208A150A1231
:1010C0000313D200080083120313CE01CC010800E1
:1010D0000800831203134C08F0007008013C031D44
:1010E0008528F101831203134B0868070318F10ADE
:1010F000CB0008304B02031D7F280730CB00FF30A8
:101100004B02031D8428CB0108007008023C031D1C
:10111000B428831203136808013C03090439043A14
:1011200003199B2851084F02013003190301FF39AD
:1011300003199B280130003C03199F28D10A680835
:10114000FF3C03090439043A0319AF28510850023F
:10115000013003190301FF390319AF280130003CA6
:101160000319B328D10308007008FF3C031D95291B
:1011700083120313CE08031DCE28F1014D08680722
:101180000318F10ACD000B3C031DC8280A30CD001E
:10119000FF304D02031DCD28CD0108004D08F100A0
:1011A0007108003C031D4E29831203134E08F20000
:1011B0007208013C031DF028F301831203133A085F
:1011C00068070318F30ABA00203C031DE928013020
:1011D000BA003A08003C031DEF281F30BA0008008F
:1011E0007208023C031D0829F301831203133B0814
:1011F00068070318F30ABB000D3C031D01290130E9
:10120000BB003B08003C031D07290C30BB00080055
:101210007208033C031D1F29F301831203133C08CA
:1012200068070318F30ABC00203C031D1829BC0101
:101230003C08FF3C031D1E291F30BC00080072083B
:10124000043C031D3629F301831203133D0868078C
:101250000318F30ABD00183C031D2F29BD013D08EA
:10126000FF3C031D35291730BD0008007208053CFE
:10127000031D4D29F301831203133E086807031869
:10128000F30ABE003C3C031D4629BE013E08FF3C5C
:10129000031D4C293B30BE00080095297108013C14
:1012A000031D5B29F2018312031349086807031821
:1012B000F20AC90095297108023C031D60298229A0
:1012C0007108033C031D652982297108043C031D34
:1012D0006A2982297108053C031D6F29822971083A
:1012E000063C031D742982297108073C031D7929D6
:1012F00082297108083C031D7E2982297108093C56
:10130000031D9429F201520868070318F20AD2005B
:101310001F3C031D8D292030D20052087B3C031D49
:1013200095297A30D20095299529962908008312AB
:101330000313690803178D0083168C130C14831292
:101340000C080800831203136A0803178D000313A7
:101350006B0803178C0003130D12831603178C13ED
:101360000C158B1355308D00AA308D008C14831210
:1013700003130D081039003C0319B729C029B729F8
:10138000831603170C110800831203136D0803174B
:101390008D0003136C0803178F0083168C170C1431
:1013A0000000000083120E080313A90003170C08A5
:1013B0000313AA00080083120313EE016F0803173A
:1013C0008F00831603132008831203178D00031365
:1013D0006E08EE0A293E8400831300088312031767
:1013E0008E0003136E08EE0A293E84008313000862
:1013F000831203178C0083168C170C158B13553032
:101400008D00AA308D008C14000000000C11831296
:101410008D0A0D080339003C031D0F2A102AE72905
:101420000800F2013030F3008316031321080F394E
:1014300073070318F20A8312B100F2013030F3008F
:1014400083162108F400F40CF40CF40C740C0F391E
:101450000F3973070318F20A8312B20008008316CB
:101460000313A2012308633C03183A2A64302302C1
:10147000A300322A2308093C0318432AA20A0A308F
:101480002302A3003A2A2208F200720EF039F03942
:10149000A200F201220823070318F20AA2000800A2
:1014A000831603132408C73C0318582A02345F2A02
:1014B0002408633C03185E2A01345F2A00340800C4
:1014C000013083160313A8008A110A1245208A15D9
:1014D0000A120800831603132508003C0319782A12
:1014E0000F30A8008A110A1245208A150A12812A93
:1014F0000C3083160313A8008A110A1245208A159E
:101500000A120800831603132708003C03198E2AC9
:10151000F2012608403E0318F20AA6002608803889
:10152000A600A8008A110A1245208A150A1208008E
:10153000FF3083120313C3008A110A126F208A1529
:101540000A1230308316A9008A110A1248208A151F
:101550000A12283083120313C3008A110A126F2063
:101560008A150A1230308316A9008A110A124820FF
:101570008A150A12303083160313A9008A110A1241
:1015800048208A150A12203083160313A9008A11F5
:101590000A1248208A150A12013083160313A80084
:1015A0008A110A1245208A150A1228308316A800CB
:1015B0008A110A1245208A150A1208308316A800DB
:1015C0008A110A1245208A150A1206308316A800CD
:1015D0008A110A1245208A150A1203308316A800C0
:1015E0008A110A1245208A150A120C308316A800A7
:1015F0008A110A1245208A150A1208008A110A1255
:101600005A208A150A12281E082B831286140B2BC7
:101610008312031386108316A81E112B831206143F
:10162000142B8312031306108316281F1A2B831200
:1016300007171D2B8312031307138316A81F232BD1
:1016400083128716262B83120313871206150000B8
:1016500006118316281C2F2B83128614322B83121B
:10166000031386108316A81C382B831206143B2BF9
:101670008312031306108316281D412B83120717AC
:10168000442B8312031307138316A81D4A2B8312BE
:1016900087164D2B831203138712061500000611BF
:1016A0008610061007138712080083160313291EDD
:1016B0005C2B831286145F2B831203138610831610
:1016C000A91E652B83120614682B831203130610C0
:1016D0008316291F6E2B83120717712B8312031396
:1016E00007138316A91F772B831287167A2B831271
:1016F000031387120615000006110A30C3008A1171
:101700000A126F208A150A1208008A110A125A203A
:101710008A150A122A1E8F2B83128614922B83128B
:10172000031386108316AA1E982B831206149B2B74
:1017300083120313061083162A1FA12B8312071787
:10174000A42B8312031307138316AA1FAA2B831239
:101750008716AD2B83120313871206160615000099
:10176000061183162A1CB72B83128614BA2B8312F8
:10177000031386108316AA1CC02B83120614C32BD6
:1017800083120313061083162A1DC92B8312071711
:10179000CC2B8312031307138316AA1DD22B83129B
:1017A0008716D52B83120313871206150000061126
:1017B00006128610061007138712080083160313FB
:1017C000AB012E082B020318FA2B2D088312E90017
:1017D0008A110A1224208A150A1283160313AC00F8
:1017E000AA008A110A124B208A150A128316AD0A22
:1017F000AB0AE12B0800831603132F08A3008A11FC
:101800000A1233208A150A12A1008A110A12302006
:101810008A150A1232088316AA008A110A124B206E
:101820008A150A1231088316AA008A110A124B205F
:101830008A150A120800831603133008A4008A11BF
:101840000A1236208A150A12A1008A110A123020C3
:101850008A150A1231088316AA008A110A124B202F
:101860008A150A1283163008A3008A110A1233203F
:101870008A150A12A1008A110A1230208A150A124A
:1018800032088316AA008A110A124B208A150A12FE
:1018900031088316AA008A110A124B208A150A12EF
:1018A000080083160313B201831603133208F900EC
:1018B000831242088A110A1293208A150A1283168B
:1018C0000313B100B20AB1080130031D0301003C4B
:1018D00003196B2C752C831603133108AA008A1187
:1018E0000A124B208A150A12542C0800831603137F
:1018F0008614061407178716831206128615061516
:10190000000007088316B3008312061100000615B5
:1019100000000611831633082039003C031D912C6A
:10192000922C7C2C831286118316861006100713C6
:101930008712080083120313D501061FA02C55142B
:10194000861FA32CD5140800831203130608203920
:101950008316B40083125602031DAF2C0034831685
:1019600034088312D600831634080319B92C0034C6
:10197000BA2C013408008312031355088316B500EE
:101980008312D501061FC52C5514861FC82CD514EB
:101990008316350883125502031DCF2C0034013005
:1019A0005502031DD42C003402305502031DD92CDE
:1019B000003483163508003C0319E52C3508033C38
:1019C00003090439043A0319E62C0130003C0319D9
:1019D000EA2C00343508831255060139003C0319FE
:1019E000F32CFF34F42C013408008A110A127520FC
:1019F0008A110A1278208A150A12D0308316B8008C
:101A00008A110A1287208A150A128316B8018A11D0
:101A10000A1287208A110A127B208A150A12D130F5
:101A20008316B8008A110A1287208A110A128A20A6
:101A30008A150A127F39C6008A110A128D208A156A
:101A40000A12B6008A110A1281208A110A128A200B
:101A50008A150A12C6008A110A128D208A150A12E6
:101A6000B5008A110A1281208A110A128A208A1569
:101A70000A12C6008A110A128D208A150A12B400B1
:101A80008A110A1281208A110A128A208A110A12E6
:101A900081208A110A128A208A150A12C6008A1128
:101AA0000A128D208A150A12B7008A110A128120A3
:101AB0008A110A128A208A150A12C6008A110A128D
:101AC0008D208A150A12B8008A110A1281208A1103
:101AD0000A128A208A150A12C6008A110A128D205B
:101AE0008A150A12B9008A110A1281208A110A1273
:101AF0008A208A110A1284208A110A127E208A15ED
:101B00000A1208008A110A1275208A110A12782016
:101B10008A150A12D0308316B8008A110A1287205B
:101B20008A150A128316B8018A110A1287208A15AB
:101B30000A123608C7008A110A1290208A150A1262
:101B40007F398316B8008A110A1287208A150A1273
:101B50003508C7008A110A1290208A150A128316C6
:101B6000B8008A110A1287208A150A123408C700A1
:101B70008A110A1290208A150A128316B8008A1157
:101B80000A1287208A150A128316B8018A110A12CE
:101B900087208A150A123708C7008A110A12902076
:101BA0008A150A128316B8008A110A1287208A152C
:101BB0000A123808C7008A110A1290208A150A12E0
:101BC0008316B8008A110A1287208A150A1239086A
:101BD000C7008A110A1290208A150A128316B800CB
:101BE0008A110A1287208A150A128316B8018A11EF
:101BF0000A1287208A110A127E208A150A1208000A
:101C0000FA3083120313C3008A110A126F208A1557
:101C10000A12FA30C3008A110A126F208A150A12BA
:101C2000FA30C3008A110A126F208A150A12FA309C
:101C3000C3008A110A126F208A150A12C50B002EE2
:101C400008008E3083120313C4000000000000005F
:101C5000000000000000C40B272E0000C30B212E43
:101C6000000008000930FD007B08FB010310FB0C9D
:101C7000FC0C0318FB07FD0B372E7B0808008312B2
:101C80000313941218309400831691010A309300C4
:101C90008715071694131413831294168C110800D9
:101CA000831603131114831203130C080839003C24
:101CB000031D5B2E532E8C11080083160313911401
:101CC000831203130C080839003C031D682E602E94
:101CD0008C110800831603131115831203130C08CB
:101CE0000839003C031D752E6D2E8C1108008316DB
:101CF000031391121116831203130C080839003CC8
:101D0000031D832E7B2E8C1108008316031391165E
:101D10001116831203130C080839003C031D912E81
:101D2000892E8C1108008316031338088312930040
:101D30000C080839003C031D9E2E982E8C110800BB
:101D4000831603139115831203130C080839003C02
:101D5000031DAB2EA32E8C1113080800831203134E
:101D6000460E0F39F000700770077007F007F00D8E
:101D7000701046080F397007080083120313470CD0
:101D8000F100710C3F394707F100710C7F394707AB
:101D9000F100710C7F39F100F10C710C3F394707EC
:101DA000F100710C7F394707F100710E0F39F10016
:101DB000F200F20D720DFC397107F200720DFE395E
:101DC0004702F200710EF039720708000E308A00E7
:101DD000EE30790703188A0A7908820754344F34A1
:101DE000423449344B347334203446346C346934CF
:101DF0006734683474344C346F34673400340F30D3
:101E00008A000730790703188A0A7908820728347C
:101E1000633429343234303430343534203431347E
:101E20002E34303432342E343034303434340034C0
:101E30000F308A002030790703188A0A7908820750
:101E400045346434693474342034503469346C3427
:101E50006F3474342034203420342034203420343F
:101E600000340F308A003930790703188A0A79085C
:101E7000820720342034203420342034203420348D
:101E800020342034203420342034203420342034B2
:101E9000203400340F308A005230790703188A0A40
:101EA00079088207453469346E3473347434653488
:101EB0006C346C3475346E34673465346E3420346D
:101EC0002034203400340F308A006B307907031837
:101ED0008A0A790882077634653472346C34613446
:101EE0007334733465346E34203420342034203419
:101EF00020342034203400340F308A0084307907B5
:101F000003188A0A790882074434613474347534BA
:101F10006D342034653469346E347334743465340C
:101F20006C346C3465346E3400340F308A009D306C
:101F3000790703188A0A79088207533463346834AE
:101F4000773465346C346C346534203453347034F5
:101F50006534653464342034203400340F308A0012
:101F6000B630790703188A0A7908820753346F3428
:101F70006C346C343A3420342034203420344934E6
:101F8000733474343A3420342034203400340F3025
:101F90008A00CF30790703188A0A7908820720342B
:101FA00046344C3449344534473445344E34003497
:101FB0000F308A00E030790703188A0A790882070F
:101FC000203420345034413452344B3445344E3470
:021FD0000034DB
:02400E00713F00
:1042000054004F00420049004B002E002E002E00AB
:1042100054004B002B0047004100530054002E0077
:1042200042004F0052004300480045005200540035
:10423000420050002B0047004100530054002E0064
:1042400054004B002B00420050002E002E002E0088
:1042500036002E002D00500049004C004F00540045
:1042600037002E002D00500049004C004F00540034
:1042700038002E002D00500049004C004F00540023
:1042800000000000400000000000000000000000EE
:00000001FF
